:0E000000802EFF022415FFFFFFFFFF0221B13B
:0300230002024D89
:20002E000B087581327508FF7509BF90A982E4F0123D6C80ED12001B80FBC82581C822C93E
:20004E002581C97A0022D083D082CF2581F581CFC082C08322CF2581F581CF22FBE0CB22DD
:20006E00FCE0FBA3E0CC22FAE0F9A3E0CA2229F9E5F03AFA227C00CB30E7011CCB2275F0CE
:20008E000030E70215F022FDE493A3FEE493A3FF4E7009E493FE740193FF800BE493A3B547
:2000AE00050BE493B5F0068F838E82E473A380D8FEEBA4FD8EF0ECA4FCEB8EF0A4C5F02C0A
:2000CE002DC5F02211D88EF0ED22C002C001AAF0F97E007D007F11C3E933F9EA33FADF0821
:2000EE00F5F0E9D001D00222ED33FDEE33FEC3ED9BF5F0EE9C40E0ADF0FED380DBBB0001C4
:20010E0022C333C5F033C5F0DBF722BB000122C3C5F013C5F013DBF722240280022401C571
:20012E00F03400C5F022C394028003C39401C5F09400C5F0223139F4C5F0F4C5F02245F04F
:20014E0070220422319B4024801A319B401E7014801A319B400E7014800A319B500E8004F1
:20016E0031AF6008E4F5F02231AF60F8E4F5F0042231AF40F780ED31AF40F170E780ED318D
:20018E00AF40E170E780DD31AF50E180D7C39BC5F09C20E70720D207C345F02220D2F9D3D7
:2001AE0022C5F0C39C7003E5F09B2290A982E0A360EEE0FFA3E0A3CF2582F582EF3583F5DC
:2001CE008380EB7E00CF2508F582EE3509F583EF227E00CF2508F9EE3509FAEF227E00C590
:2001EE00082FC508C5093EC50922E4F50AA88108E4F608B880FB22E4F520D201D200D20333
:20020E00D205C2B4E4F50EF50DF50CF50BE4F512F511F510F50F74FFF513E588543FF588A7
:20022E00E589540FF5894420F5897450F598E5874480F58774FAF58BF58DD28ED2AC22C052
:20024E00E0C0D0C083C082309839E50DB4FA028030502E050DE50DB50E0280044002F50E38
:20026E0090A000C0E0E50B2582F582E43583F583D0E0E599F0050BE50BB4FA004003750BEF
:20028E0000C298309948E511700DD200300235E4D5E0FDC2B4802DC20030011A300202D26D
:2002AE00B490A0FAC0E0E5102582F582E43583F583D0E0E0F59915110510E510B4FA00404F
:2002CE0003751000C299200105200002D299D082D083D0D0D0E0322278FB120048E6C0E0DE
:2002EE00B40A0B300308D204740D1581C0E0E511B4FA0280F950F7C2AC90A0FAC0E0E50FCD
:20030E002582F582E43583F583D0E0D0E0C0E0F00511050FE511B512004002F512E50FB4D5
:20032E00FA004003750F00300002D299D2ACD0E0300408C204740AC0E080B322E4F5F0786D
:20034E00FB120048F608A6F022E51364FF7038E50D6034300531C2AC90A000C0E0E50C2541
:20036E0082F582E43583F583D0E0E0D2ACB40A0302038574018010150D050CE50CB4FA0032
:20038E004003750C0080C875F00022E4A20192E0F51F70030203BAE51160030203A5E4A2F4
:2003AE000092E0F51FE51F70030203AC22C2AC7513FF7400F50CF50BC50DD2AC75F000221E
:2003CE0074FFC513B4FF2EE50D0060FBC2AC90A000C0E0E50C2582F582E43583F583D0E085
:2003EE00E0C0E0150D050CE50CB4FA004003750C00D2ACD0E030050BB40A030203D5B40D0F
:20040E0002740A75F000221203CEC0E0C0E0C0E01202E6D0E0D0E0D0E075F00022E5137506
:20042E00F0007BFF7C0012016E700302044374FFF5F002045378FB120048E60886F0F513A1
:20044E0018E60886F02278FB1200488682088683E06016C083C082C0E0C0E01202E6D0E045
:20046E00D0E0D082D083A380E722E4F5F078FB120048F608A6F022745E75F042C0E0C0F0D8
:20048E00E52075F000C0E0C0F07402123E341581158115811581747975F042C0E0C0F0E579
:2004AE000F75F000C0E0C0F0E510C0E0C0F0E51175F000C0E0C0F0E512C0E0C0F074057545
:2004CE00F000123E347FF612005474AC75F042C0E0C0F0E50B75F000C0E0C0F0E50CC0E072
:2004EE00C0F0E50D75F000C0E0C0F0E50EC0E0C0F0740575F000123E347FF6120054E4F53E
:20050E000EF512227FFD7EFF1201EDE4F5F07F001201D1F0A3C5F0F0C5F078FB120048E6D1
:20052E000886F012013918F608A6F012012B45F06022181818860108860289828A831200B9
:20054E007589828A83E012008CC0E0C0F0123F2D1581158145F0700302061E7F001201D157
:20056E00E0A3F5F0E0C5F07B047C0012010B7F001201D1F0A3C5F0F0C5F078F912004886B6
:20058E000108860289828A8312007589828A83E012008CC0E0C0F0123F3C158115817F02FD
:2005AE001201D1F07F021201D1E012008C7B39120083120158600B7F021201D1E0C394308B
:2005CE00800B7F021201D1E0C39441240A75F0007F001201D112006E2BC5F03CC5F07F00DF
:2005EE001201D1F0A3C5F0F0C5F078F9120048860108860289828A83E0A3F5F0E0C5F01213
:20060E00012B89828A83F0A3C5F0F0C5F00205287F001201D1E0A3F5F0E0C5F07F03020187
:20062E00EB7FF17EFF1201ED7F021201DFE98AF0C0E0C0F0E4C0E0C0E0740A75F000C0E007
:20064E00C0F0123F6E7FFA1200547F021201DFE98AF07F0C1201D1F0A3C5F0F0C5F074098F
:20066E007F0E1201D1F078FB120048860108860289828A8312007589828A83E012008CC032
:20068E00E0C0F0123EF41581158145F0602E78FB120048860108860289828A83120075897D
:2006AE00828A83E012008CC0E0C0F0123F281581158145F060067F0E1201D1E070030207C2
:2006CE003E7F0C1201D1E0A3F5F0E0C5F012012B7F0C1201D1F0A3C5F0F0C5F0120139F983
:2006EE00AAF0C001C00278F9120048860108860289828A8312007589828A83E0D083D082B1
:20070E00F018860108860289828A83E0A3F5F0E0C5F012012B89828A83F0A3C5F0F0C5F054
:20072E007F0E1201D1E0147F0E1201D1F00206747F021201DFE98AF0C0E0C0F0123F91154C
:20074E008115817F001201D1F0A3C5F0F0C5F07F0F0201EB7FFE7EFF1201EDE4F5F07F0066
:20076E001201D1F0A3C5F0F0C5F07F001201D1E0A3F5F0E0C5F012014C45F0601B78FB12A6
:20078E000048E60886F012013918F608A6F012012B7B007C0012016045F0700302080878CD
:2007AE00F7120048E60886F012012B18F608A6F0120139F9AAF089828A83E012008CC0E077
:2007CE00C0F008E60886F012012B18F608A6F0120139F9AAF089828A83E012008CFBACF0F9
:2007EE00D0F0D0E0C39BC5F09CC5F07F001201D1F0A3C5F0F0C5F00207787F001201D1E003
:20080E00A3F5F0E0C5F07F020201EB7FFF7EFF1201EDE47F001201D1F07F001201D1E07554
:20082E00F0007B107C0012018570120208887F001201D1E0047F001201D1F080DC78FB128C
:20084E000048E60886F07F001201D112006A2BC5F03400C5F0F9AAF07F001201D1E0C0019F
:20086E00C00279567AA412008C12007C89828A83E0F4D083D082F002083C740190A47AF0B5
:20088E007F010201EB7FFF7EFF1201EDE4F521E4F5F090A2BEF0A3C5F0F0C5F0E490A2BD6E
:2008AE00F074F475F0A1C0E0C0F0E4C0E0C0E074C975F000C0E0C0F0123F6E7FFA120054C8
:2008CE00E4F5F090A389F0A3C5F0F0C5F074C075F0A2C0E0C0F0E4C0E0C0E074C975F00047
:2008EE00C0E0C0F0123F6E7FFA120054E490A455F0748C75F0A3C0E0C0F0E4C0E0C0E074AF
:20090E00C975F000C0E0C0F0123F6E7FFA120054740190A47AF0E47F001201D1F07F0012D2
:20092E0001D1E075F0007B107C0012017F70120209997F001201D1E0047F001201D1F080B9
:20094E00DC7F001201D1E079567AA412008C12007C7F001201D1E0C001C00279687AA4127A
:20096E00008C12007C89828A83E0F412008CD083D08212006A120083120176700302099672
:20098E00E490A47AF002099902094090A47AE060030209DE745675F0A4C0E0C0F0E4C0E057
:2009AE00C0E0741275F000C0E0C0F0123F6E7FFA120054745675F0A4C0E0C0F0745775F05D
:2009CE0042C0E0C0F0123FDA158115811581158112175B1217F5746875F0A4C0E0C0F0120B
:2009EE000819158115817F010201EB12039978FB120048E60886F090A38BF0C209C2B490D0
:200A0E00A38BE075F000900A37020095E490A38BF0D208C202E490A981F0020A4BC208D23C
:200A2E0002E490A981F0020A4B2B0A03002B0A02002B0A01001F0A000000001A0A227FFB33
:200A4E007EFF1201ED78F9120048E60886F07F031201D1F0A3C5F0F0C5F008E60886F07F9E
:200A6E00011201D1F0A3C5F0F0C5F07F011201DFE98AF0C0E0C0F0740275F000C0E0C0F046
:200A8E0012051215811581158115817F001201D1F078FB120048E60886F0C0E0C0F074304F
:200AAE0075F000C0E0C0F07402C0E0C0F0123F6E7FFA1200547F031201D112007589828A8D
:200ACE0083E07003020B0F7F031201D11200757F001201D1E089828A8312006A2B7F001296
:200AEE0001D1F07F031201D1E0A3F5F0E0C5F012012B7F031201D1F0A3C5F0F0C5F0020A26
:200B0E00C37F001201D1E0F4047F001201D1F078FB12004886010886027F001201D1E075DA
:200B2E00F0007B047C00120119C001C00290425C12007512007C89828A83E0D083D082F03D
:200B4E0078FB120048E60886F02401C5F03400C5F0F9AAF07F001201D1E0540FC001C002D7
:200B6E0090425C12007512008C12007C89828A83E0D083D082F07F001201D1E012008C54C4
:200B8E00FFC5F05400C5F07F050201EB90A455E06003020C40748C75F0A3C0E0C0F0E4C002
:200BAE00E0C0E074C975F000C0E0C0F0123F6E7FFA12005490A38BE075F0007B007C00120B
:200BCE00018D7003020C2C798C7AA3742489828A83F0E4A20992E0F51F748C75F0A3C0E04D
:200BEE00C0F0E51F600774F075F042800574F475F042C0E0C0F0123FCA15811581158115EB
:200C0E0081748C75F0A3C0E0C0F0745675F0A4C0E0C0F0123FCA1581158115811581748C57
:200C2E0075F0A3C0E0C0F01240081581158190A455F078FB120048E60886F07B0A7C00120B
:200C4E00016E700C18E60886F07BFF7C0012016E45F07003020CD1E4A20992E0F51F700399
:200C6E00020C94748C75F0A3C0E0C0F0748C75F0A32401C5F03400C0F0C0E0120A4C158108
:200C8E00158115811581748C75F0A3C0E0C0F01204541581158178FB120048E60886F07BEA
:200CAE000A7C0012016E7003020CC9740A75F000C0E0C0F01202E615811581E490A455F01F
:200CCE00020CFD748C75F0A390A45512006A2BC5F03400C5F0F9AAF078FB120048E6088651
:200CEE00F089828A83F090A455E00490A455F02278FB120048860108860289828A83E0709A
:200D0E0003020D3F18860108860289828A83E012008CC0E0C0F0120B9A1581158178FB12F7
:200D2E000048E60886F012012B18F608A6F0020CFE227FFA7EFF1201EDE4F5F07F0212018E
:200D4E00D1F0A3C5F0F0C5F078FB120048E60886F07F001201D1F0A3C5F0F0C5F0E47F04DF
:200D6E001201D1F07F041201D1E075F0007B027C0012017F7003020FC07F041201D1E0755A
:200D8E00F000900F96020095C2097F001201D1E0A3F5F0E0C5F012012B7F001201D1F0A32A
:200DAE00C5F0F0C5F0120139F9AAF089828A83E012008C900F0D0200957F001201D112009E
:200DCE007589828A83E012008C7B2012008312016E7003020DEF74017F041201D1F0020DFD
:200DEE00F774037F041201D1F0020F1978FB120048E60886F0C0E0C0F018E60886F02401D4
:200E0E00C5F03400C0F0C0E0120A4C15811581158115817F051201D1F07F051201D1E070BB
:200E2E0003020EAD74037F041201D1F0742F75F075C0E0C0F090A2BEE0A3F5F0E0C5F0124A
:200E4E00012B90A2BEF0A3C5F0F0C0F0C0E012404F158115811581158190A2BEF0A3C5F0AF
:200E6E00F0C5F090A38BE075F0007B027C0012016E7003020EAA74F675F042C0E0C0F07F35
:200E8E00051201D1E075F000C0E0C0F0740275F000123E341581158115811581020EFF7F81
:200EAE00001201D1E0A3F5F0E0C5F02402C5F03400C5F07F001201D1F0A3C5F0F0C5F07FB0
:200ECE00001201D112007589828A83E012008C7B2012008312016E7003020EF774017F04E0
:200EEE001201D1F0D209020EFF74037F041201D1F0020F1974037F041201D1F0020F19FA3C
:200F0E000D2300C70D21000000020F020FA2745675F0A4C0E0C0F07F001201D1E0A3F5F0EC
:200F2E00E0C0F0C0E0745675F0A4C0E0C0F012400815811581C0E0C0F01207627FFA120074
:200F4E005445F07003020F6174037F041201D1F0020F9374027F041201D1F0745675F0A403
:200F6E00C0E0C0F0124008158115817F001201D112006E2BC5F03CC5F07F021201D1F0A3E1
:200F8E00C5F0F0C5F0020FA21C0F0100960D00000000A20F7F001201D1E0A3F5F0E0C5F056
:200FAE0012012B7F001201D1F0A3C5F0F0C5F0020D727F021201D1E0A3F5F0E0C5F07F062D
:200FCE000201EB7FFD7EFF1201EDE4F5F07F011201D1F0A3C5F0F0C5F012035745F07003EE
:200FEE000212741203CE7F001201D1F0E4A20892E0F51F700302101A7F001201D1E012001D
:20100E008CC0E0C0F01202E61581158190A2BDE0600302104274F475F0A1C0E0C0F0E4C0D8
:20102E00E0C0E074C975F000C0E0C0F0123F6E7FFA1200547F001201D1E012008C9010BA57
:20104E0002009590A2BDE0700302107390A2BDE01490A2BDF079F47AA112008C12007CE4CA
:20106E0089828A83F00210C60210C674F475F0A190A2BD12006A2BC5F03400C5F0F9AAF075
:20108E007F001201D1E089828A83F090A2BDE00490A2BDF075F0007BC87C00120195700306
:2010AE000210B774C790A2BDF00210C676100A0051100800000079107F001201D1E0120090
:2010CE008C7B0A12008312016E700302127490A38BE075F00090125B02009579F47AA18938
:2010EE00828A83E012008C7B2A120083120176700302111374F475F0A17F011201D1F0A314
:20110E00C5F0F0C5F002126F74F475F0A1C0E0C0F0120D40158115817F011201D1F0A3C5DF
:20112E00F0F0C5F002126F90A2BDE070030211B279F47AA189828A83E012008C9011A2021F
:20114E0000950211B2740D75F043C0E0C0F01204541581158174F475F0A1C0E0C0F0120444
:20116E005415811581740F75F043C0E0C0F01204541581158174F475F0A1C0E0C0F0120DF3
:20118E0040158115817F011201D1F0A3C5F0F0C5F00211B250112D0050112A005011240021
:2011AE000000531102126F90A2BDE0700302124579F47AA189828A83E012008C90123502A8
:2011CE00009502124574F475F0A1C0E0C0F0120D40158115817F011201D1F0A3C5F0F0C569
:2011EE00F07F011201D1E0A3F5F0E0C5F045F07003021232741175F043C0E0C0F0120454BB
:20120E0015811581745675F0A4C0E0C0F012045415811581741575F043C0E0C0F0120454F0
:20122E0015811581021245D0112D00D0112A00D01124000000D31102126F740175F000C0FC
:20124E00E0C0F01209F91581158102126FB51103003511020016110100E9100000000048B3
:20126E0012E490A2BDF07F011201D1E0A3F5F0E0C5F07F030201EB90A38BE075F0007B003C
:20128E007C0012016E700E90A38BE075F0007B027C0012016E45F070030212BE78FB120049
:2012AE0048E60886F0C0E0C0F0120CFE158115812290A38BE075F0007B007C0012016E70CF
:2012CE00030212F2745675F0A4C0E0C0F012045415811581741975F043C0E0C0F01204544F
:2012EE0015811581227FFD7EFF1201ED78FB120048E60886F02401C5F03400C5F0F9AAF012
:20130E0089828A83E012008C7B3D12008312016E700302144E18E60886F02402C5F03400F9
:20132E00C5F07F001201D1F0A3C5F0F0C5F07F001201D1E0A3F5F0E0C0F0C0E01240081530
:20134E008115817B017C00120168700302143B745675F0A4C0E0C0F0E4C0E0C0E0741275EF
:20136E00F000C0E0C0F0123F6E7FFA120054E47F021201D1F07F021201D1E075F0007B1013
:20138E007C0012017F600D7F001201D112007589828A83E070120213F87F021201D1E0040A
:2013AE007F021201D1F080CD7F021201D1E079567AA412008C12007C7F001201D1E0A3F544
:2013CE00F0E0C5F012012B7F001201D1F0A3C5F0F0C5F0120139C001C002F9AAF089828AF5
:2013EE0083E0D083D082F00213A7745675F0A4C0E0C0F0745675F0A4C0E0C0F01240081576
:20140E00811581D004D0032BC5F03CC5F0F9AAF0742089828A83F012175B746875F0A4C0D7
:20142E00E0C0F01208191581158102144B741B75F043C0E0C0F01212851581158102149943
:20144E0012175B746875F0A4C0E0C0F01208191581158174C075F0A2C0E0C0F0743575F0CD
:20146E0043C0E0C0F0745675F0A4C0E0C0F0740375F000123E457FFA12005474C075F0A21D
:20148E00C0E0C0F0120CFE158115817F030201EB78FB120048E60886F018F608A6F074C025
:2014AE0075F0A2C0E0C0F0744875F043C0E0C0F0745675F0A4C0E0C0F0740375F000123EC4
:2014CE00457FFA12005474C075F0A2C0E0C0F0120CFE15811581788018E660FC881F74C0DA
:2014EE0075F0A2C0E0C0F0745975F043C0E0C0F0E51F75F000C0E0C0F0747FC0E0C0F07452
:20150E000475F000123E457FF812005474C075F0A2C0E0C0F0120CFE158115812278FB1268
:20152E000048E60886F018F608A6F074C075F0A2C0E0C0F0747375F043C0E0C0F0E50A7577
:20154E00F000C0E0C0F090A2BEE0A3F5F0E0C0F0C0E0740475F000123E457FF812005474F2
:20156E00C075F0A2C0E0C0F0120CFE15811581E4F50AE4F5F090A2BEF0A3C5F0F0C5F02253
:20158E007FFE7EFF1201ED78FB120048E60886F02401C5F03400C5F07F001201D1F0A3C594
:2015AE00F0F0C5F07F001201D112007589828A83E012008CC0E0C0F0123F281581158145CE
:2015CE00F070030215F07F001201D1E0A3F5F0E0C0F0C0E0123F911581158190A981F002DE
:2015EE00162A74C075F0A2C0E0C0F074A275F043C0E0C0F090A981E075F000C0E0C0F07441
:20160E000375F000123E457FFA12005474C075F0A2C0E0C0F0120CFE158115817F02020189
:20162E00EB7FFE7EFF1201ED78FB120048E60886F02401C5F03400C5F07F001201D1F0A3CD
:20164E00C5F0F0C5F07F001201D112007589828A83E012008C9016FE02009574C075F0A22C
:20166E00C0E0C0F074B675F043C0E0C0F090A38BE075F000C0E0C0F0740375F000123E4526
:20168E007FFA12005474C075F0A2C0E0C0F0120CFE158115810217067F001201D112007581
:2016AE0089828A83E012008CC0E0C0F0123F281581158145F070030216EB7F001201D1E0A3
:2016CE00A3F5F0E0C0F0C0E0123F9115811581C0E0C0F01209F9158115810216FB74C675E4
:2016EE00F043C0E0C0F012128515811581021706691600000000A6167F020201EB90A38BFD
:20170E00E075F0007B007C0012016E700302175A74C075F0A2C0E0C0F074DE75F043C0E0F3
:20172E00C0F078F7120048E60886F0C0E0C0F0740375F000123E457FFA12005474C075F085
:20174E00A2C0E0C0F012128515811581227FFD7EFF1201EDE590F4540E12008C7B011200A2
:20176E00831201197F001201D1F07F001201D1E044307F011201D1F0745675F0A4C0E0C01B
:20178E00F0124008158115817F021201D1F07F021201D1E075F0007B027C001201957003B2
:2017AE000217D27F021201D1E0C3940279567AA412008C12007C7F011201D1E089828A831D
:2017CE00F00217E7E4F5F079567AA412007C7F011201D1E089828A83F07F001201D1E01226
:2017EE00008C7F030201EBD290E4A29092E0F51F7003021816740175F000C0E0C0F01209F9
:20180E00F915811581021822E4C0E0C0E01209F915811581227FFA7EFF1201ED78FB120058
:20182E0048E60886F07F021201D1F0A3C5F0F0C5F07F001201D1F0A3C5F0F0C5F07F0012BB
:20184E0001D112007589828A83E070030218FD7F001201D112007589828A83E012008C7BA4
:20186E002012008312016E70030218987F001201D1E0A3F5F0E0C5F012012B7F001201D1FE
:20188E00F0A3C5F0F0C5F00218FA7F021201D1120075C001C0027F001201D11200758982D5
:2018AE008A83E012008CC0E0C0F0123F3C15811581D083D082F07F001201D1E0A3F5F0E046
:2018CE00C5F012012B7F001201D1F0A3C5F0F0C5F07F021201D1E0A3F5F0E0C5F012012B17
:2018EE007F021201D1F0A3C5F0F0C5F002184B7F021201D1120075E489828A83F078FB12C6
:20190E000048E60886F02401C5F03400C5F07F001201D1F0A3C5F0F0C5F0188601088602CB
:20192E0089828A83E012008C90209902009578FB120048E60886F0C0E0C0F01212F31581F5
:20194E0015810220D97F001201D112007589828A83E012008CC0E0C0F0123F281581158173
:20196E0045F070030219917F001201D1E0A3F5F0E0C0F0C0E0123F911581158190A50AF0CD
:20198E000219CB74C075F0A2C0E0C0F074F975F043C0E0C0F090A50AE075F000C0E0C0F08F
:2019AE00740375F000123E457FFA12005474C075F0A2C0E0C0F0120CFE158115810220D9FB
:2019CE007F001201D112007589828A83E012008C901A4D0200957F001201D1E0A3F5F0E040
:2019EE00C5F02401C5F03400C0F0C0E0123F9115811581C0E0C0F012325C15811581021A80
:201A0E00597F001201D1E0A3F5F0E0C5F02401C5F03400C0F0C0E0123F9115811581C0E0F3
:201A2E00C0F0122F6415811581021A59741B75F044C0E0C0F012128515811581021A590FC1
:201A4E001A5400E419520000003A1A0220D912149E122C3C123CFF0220D978FB120048E633
:201A6E000886F0C0E0C0F012152B158115810220D97F001201D112007589828A83E012001D
:201A8E008CC0E0C0F0123F281581158145F07003021B197F001201D1E0A3F5F0E0C0F0C0BE
:201AAE00E0123F911581158190A97BF0A3C5F0F0C5F07B147C0012017F7003021B167414BE
:201ACE0075F00090A97BF0A3C5F0F0C5F074C075F0A2C0E0C0F0743675F044C0E0C0F09034
:201AEE00A97BE0A3F5F0E0C0F0C0E0740375F000123E457FFA12005474C075F0A2C0E0C031
:201B0E00F012128515811581021B5474C075F0A2C0E0C0F0745F75F044C0E0C0F090A97B76
:201B2E00E0A3F5F0E0C0F0C0E0740375F000123E457FFA12005474C075F0A2C0E0C0F01212
:201B4E000CFE158115810220D978FB120048E60886F0C0E0C0F012158E158115810220D9E9
:201B6E0078FB120048E60886F0C0E0C0F012162F158115810220D97F001201D1E0A3F5F08D
:201B8E00E0C5F02402C5F03400C5F0F9AAF089828A83E012008CC39430C5F09400C5F07FB1
:201BAE00041201D1F0A3C5F0F0C5F07F001201D1E0A3F5F0E0C5F02401C5F03400C5F0F926
:201BCE00AAF089828A83E012008C7B3D12008312016E60287F041201D1E0A3F5F0E0C5F00D
:201BEE007B007C0012016860137F041201D1E0A3F5F0E0C5F07B017C0012015845F0700383
:201C0E00021CA47F001201D112007589828A83E012008C901C910200957F041201D1E0A3B6
:201C2E00F5F0E0C5F045F07003021C3FD296021C41C296021CA17F041201D1E0A3F5F0E08A
:201C4E00C5F045F07003021C5CD295021C5EC295021CA17F041201D1E0A3F5F0E0C5F045FD
:201C6E00F07003021C79D294021C7BC294021CA1748375F044C0E0C0F01212851581158183
:201C8E00021CA1611C4300441C4200271C410000007E1C021CB4749C75F044C0E0C0F0120A
:201CAE001285158115810220D97F001201D112007589828A83E012008CC0E0C0F0123F280F
:201CCE001581158145F07003021D087F001201D1E0A3F5F0E0C0F0C0E0123F9115811581F2
:201CEE0090A97FF0A3C5F0F0C5F0E4F5F090A97DF0A3C5F0F0C5F0021D4374C075F0A2C068
:201D0E00E0C0F074B575F044C0E0C0F090A97FE0A3F5F0E0C0F0C0E0740375F000123E4542
:201D2E007FFA12005474C075F0A2C0E0C0F0120CFE158115810220D97F001201D1120075FE
:201D4E0089828A83E07003021E7C7F001201D1E0A3F5F0E0C0F0C0E0742D75F000C0E0C00D
:201D6E00F012409615811581158115817F021201D1F0A3C5F0F0C5F07F021201D1E0A3F5F6
:201D8E00F0E0C5F07B007C0012016E7003021E1E7F001201D112007589828A83E012008C07
:201DAE00C0E0C0F0123F281581158145F07003021E0B7F001201D1E0A3F5F0E0C0F0C0E052
:201DCE00123F91158115817F041201D1F0A3C5F0F0C5F07F041201D1E0A3F5F0E0C0F0C074
:201DEE00E07F041201D1E0A3F5F0E0C0F0C0E012299D1581158115811581021E1B74CD75D5
:201E0E00F044C0E0C0F012128515811581021E797F001201D1E0A3F5F0E0C0F0C0E0123F76
:201E2E0091158115817F041201D1F0A3C5F0F0C5F07F041201D1E0A3F5F0E0C0F0C0E07F05
:201E4E00021201D1E0A3F5F0E0C5F02401C5F03400C0F0C0E0123F9115811581C0E0C0F0D5
:201E6E0012299D1581158115811581021E95E4C0E0C0E074FF75F001C0E0C0F012299D1535
:201E8E00811581158115810220D97F001201D1E0A3F5F0E0C0F0C0E074E475F044C0E0C09A
:201EAE00F01240B3158115811581158145F07003021ED474E975F044C0E0C0F01212851517
:201ECE00811581021EDA1203990200000220D97F001201D112007589828A83E012008CC0F8
:201EEE00E0C0F0123F281581158145F07003021F397F001201D1E0A3F5F0E0C0F0C0E01290
:201F0E003F9115811581C0E0C0F01228021581158145F07003021F3674FE75F044C0E0C085
:201F2E00F012128515811581021F49740C75F045C0E0C0F0121285158115810220D90220F8
:201F4E00D9742375F045C0E0C0F0120CFE15811581745875F045C0E0C0F0120CFE15811534
:201F6E0081747375F045C0E0C0F0120CFE15811581749575F045C0E0C0F0120CFE158115DF
:201F8E008174C175F045C0E0C0F0120CFE1581158174FB75F045C0E0C0F0120CFE1581150B
:201FAE0081743575F046C0E0C0F0120CFE15811581747075F046C0E0C0F0120CFE15811500
:201FCE0081749975F046C0E0C0F0120CFE1581158174C275F046C0E0C0F0120CFE1581152A
:201FEE008174EF75F046C0E0C0F0120CFE15811581740E75F047C0E0C0F0120CFE15811567
:20200E0081743975F047C0E0C0F0120CFE15811581746C75F047C0E0C0F0120CFE1581159D
:20202E0081749375F047C0E0C0F0120CFE1581158174BA75F047C0E0C0F0120CFE158115D5
:20204E008174EE75F047C0E0C0F0120CFE15811581740E75F048C0E0C0F0120CFE15811505
:20206E0081742D75F048C0E0C0F0120CFE158115810220D978FB120048E60886F0C0E0C05F
:20208E00F012170B158115810220D94F1F3F004C1F0000DD1E5300981E5200461D5100B70E
:2020AE001C5000851B4F006E1B4E00571B4C007F1A4900681A45005C1A4400CE1943005342
:2020CE001942003C194100000082207F060201EBC2B3E4F522E4F514E4F517747B75F0ED5E
:2020EE00F51885F019E4F51AE4F530742890A50AF0747B75F0A4C0E0C0F0E4C0E0C0E07490
:20210E002075F000C0E0C0F0123F6E7FFA120054E4F527F526F525F524749B75F0A4C0E038
:20212E00C0F0E4C0E0C0E0742075F000C0E0C0F0123F6E7FFA120054E4F52BF52AF529F5A0
:20214E0028E4F516F51574BB75F0A4C0E0C0F0E4C0E0C0E0744F75F000C0E0C0F0123F6E6D
:20216E007FFA120054740B75F0A5C0E0C0F0E4C0E0C0E0E475F004C0E0C0F0123F6E7FFAA0
:20218E00120054E58854CFF588E58954F0F5894401F589E4F58AF58CD2B9D2A9D28CD28829
:2021AE00D2A822C0E0C0D0C28C85188A85198CD28CA2149215A2B2B39214C0F0C083C08209
:2021CE00C000E514B4020280044002740075F003A49021E3730221EC02222D022277051A19
:2021EE00E53060021530E5314532600DC3E5319401F531E5329400F5322016030223FAC29B
:20220E0016751401751A007515007518BC7519FDC28C85188A85198CD28CB2970223FA902E
:20222E00A4BBE5152582F582E5833400F583E0A2E092B30515E515B5160050030223FAC24B
:20224E00B375140075187B7519EDC28C85188A85198CD28CE51675F00884251AF51A90A545
:20226E000AE0F530B2970223FA301305C2130223FAE517B40A0280044002740A75F003A491
:20228E00902292730222B30222D00222E302230402231102233A02234802235B02237C0259
:2022AE0023890223F130146D7518BC7519FDC28CE518241EF58AE43519F58CD28C0517028E
:2022CE00231EA215B014504D752C00752D007515090517803BA215B01492D5A214B015721B
:2022EE00D55032E52DA21413F52DE52C13F52CD5151E0517801AA215B01450197515020504
:20230E0017800D20150F20140CD5150405178000D2130223FA75170A0223FA75140075172F
:20232E000075187B7519EDB2970223FAA215B3821450E2751509051780D6A215B01450D5CD
:20234E00752E00752F00751509051780C3A215B01492D5A214B01572D550BAE52FA21413AB
:20236E00F52FE52E13F52ED515A6051780A2A215B01450A175150305178071201497D51559
:20238E006BE52C652E7094E52D652F708E852D83852C8275F007C3E58313F583E58213F57F
:2023AE0082D5F0F385832D85822CE52825E0249BF58274A43400F583E52CF0A3E52DF005B6
:2023CE00287410B5280280025003752800052AE52AB52B0280044002F52B7406251AF51A24
:2023EE00022329201506201403022329E51AB4C2004006D217243EF51AD000D082D083D067
:20240E00F0D0D0D0E03222C0E0C0F0C0D0C083C082E514B4020280044002740025E0902411
:20242E0030738004801F801F7518E17519FEC28C85188A85198CD28C751700751500751493
:20244E0002B297800E800CC28C758AE1758CFED28C8000D082D083D0D0D0F0D0E03222787D
:20246E00F9120048E60886F05401C5F05400C5F07B007C0012016E70030224B0088601082C
:20248E008602740189828A83F018E60886F02401C5F03400C5F0F9AAF0E489828A83F00269
:2024AE0024D778FB1200488601088602E489828A83F018E60886F02401C5F03400C5F0F90B
:2024CE00AAF0740189828A83F0227FFF7EFF1201ED740175F000C0E0C0F078F9120048E6DF
:2024EE000886F02400C5F03400C0F0C0E012246D1581158115811581E4C0E0C0E078F91251
:20250E000048E60886F02402C5F03400C0F0C0E012246D158115811581158178FB120048DA
:20252E00E60886F02404C5F03400C5F018F608A6F0E47F001201D1F07F001201D1E075F0D8
:20254E00007B097C0012017F70120225B57F001201D1E0047F001201D1F080DC78F9120004
:20256E0048E60886F0C0E0C0F008E60886F0C0E0C0F012246D158115811581158178F91217
:20258E000048E60886F07B017C0012011918F608A6F008E60886F02402C5F03400C5F01869
:2025AE00F608A6F002255BE4C0E0C0E078F9120048E60886F0C0E0C0F012246D1581158185
:2025CE00158115817F010201EB78FB120048E60886F07BFF7CFF120176600690A981E05450
:2025EE0002700302263974C075F0A2C0E0C0F0744975F048C0E0C0F078F7120048E6088675
:20260E00F0C0E0C0F018E60886F0C0E0C0F0740475F000123E457FF812005474C075F0A216
:20262E00C0E0C0F0120CFE1581158174BB75F0A4C0E0C0F0E4C0E0C0E0744F75F000C0E080
:20264E00C0F0123F6E7FFA12005478FB120048E60886F0C0E0C0F074BB75F0A42418C5F074
:20266E003400C0F0C0E01224D8158115811581158178FB120048E60886F0C0E0C0F074BBB2
:20268E0075F0A42434C5F03400C0F0C0E01224D81581158115811581744FF516D216227FD5
:2026AE00FE7EFF1201EDE52A7003022702E52975F000C333C5F033C5F0799B7AA412007C1E
:2026CE0089828A83E0A3F5F0E0C5F07F001201D1F0A3C5F0F0C5F0152A0529E529E5297589
:2026EE00F0007B107C0012019570030226FFE4F52902271274FFF5F07F001201D1F0A3C543
:20270E00F0F0C5F07F001201D1E0A3F5F0E0C5F07BFF7CFF120176600690A981E054017073
:20272E000302277D74C075F0A2C0E0C0F0745C75F048C0E0C0F07F001201D1E0A3F5F0E0DF
:20274E00C0F0C0E07F001201D1E0A3F5F0E0C0F0C0E0740475F000123E457FF8120054745D
:20276E00C075F0A2C0E0C0F0120CFE158115817F001201D1E0A3F5F0E0C5F07F020201EB1D
:20278E007FFE7EFF1201ED1226AD7F001201D1F0A3C5F0F0C5F07F001201D1E0A3F5F0E051
:2027AE00C5F07BFF7CFF12017660137F001201D1E0A3F5F0E0C5F07BFF7C0112017F45F047
:2027CE0070030227FD7F001201D1E0A3F5F0E0C5F0C333C5F033C5F0790B7AA512007C74BA
:2027EE000175F00089828A83F0A3C5F0F0C5F07F020201EB7FFE7EFF1201ED78FB1200482A
:20280E00E60886F07BFF7C01120185600CE52675F0007B107C0012017F45F07003022898D8
:20282E00E52475F000C333C5F033C5F0797B7AA412007C78FB120048E60886F089828A83A0
:20284E00F0A3C5F0F0C5F00524E524E52475F0007B107C00120195700302286DE4F5240522
:20286E0026E526E52675F000AB277C0012018D7003022886E526F527E4F5F07F001201D145
:20288E00F0A3C5F0F0C5F00228A9740175F0007F001201D1F0A3C5F0F0C5F07F001201D1DD
:2028AE00E0A3F5F0E0C5F07F020201EB7FFE7EFF1201EDE526700302290FE52575F000C3BA
:2028CE0033C5F033C5F0797B7AA412007C89828A83E0A3F5F0E0C5F07F001201D1F0A3C5AA
:2028EE00F0F0C5F015260525E525E52575F0007B107C00120195700302290CE4F5250229D5
:20290E001F74FFF5F07F001201D1F0A3C5F0F0C5F07F001201D1E0A3F5F0E0C5F07F0202FF
:20292E0001EB7FFE7EFF1201EDE53012008C12014C45F0600CE51475F0007B007C00120188
:20294E006E45F070030229981228BA7F001201D1F0A3C5F0F0C5F07F001201D1E0A3F5F081
:20296E00E0C5F07BFF7CFF12017670030229927F001201D1E0A3F5F0E0C0F0C0E01225D7FD
:20298E001581158190A50AE0F5307F020201EB7FFD7EFF1201ED78F9120048E60886F0081A
:2029AE00860308860412016E7003022A4D74C075F0A2C0E0C0F0746F75F048C0E0C0F018FE
:2029CE001818E60886F0C0E0C0F018E60886F0C333C5F033C5F0790B7AA512007C89828A30
:2029EE0083E0A3F5F0E0C5F045F06007740175F0008003E4F5F0C0E0C0F0740475F0001248
:202A0E003E457FF812005474C075F0A2C0E0C0F0120CFE1581158178F9120048E60886F046
:202A2E00C333C5F033C5F0790B7AA512007CE4F5F089828A83F0A3C5F0F0C5F0022C37741D
:202A4E00C075F0A2C0E0C0F0747975F048C0E0C0F078F5120048E60886F0C0E0C0F008E6FE
:202A6E000886F0C0E0C0F0740475F000123E457FF812005474C075F0A2C0E0C0F0120CFE84
:202A8E001581158178F9120048E60886F00886030886041201587003022C27E47F00120101
:202AAE00D1F0181818E60886F07F011201D1F0A3C5F0F0C5F078F9120048E60886F02408EF
:202ACE00C5F03400C5F07F011201D112006E12016060157F011201D1E0A3F5F0E0C5F00815
:202AEE00860308860412015845F07020022B9D7F011201D1E0A3F5F0E0C5F012012B7F0194
:202B0E001201D1F0A3C5F0F0C5F080A97F001201D1E075F0007B017C001201197F0012014F
:202B2E00D1F07F011201D1E0A3F5F0E0C5F0C333C5F033C5F0790B7AA512007C89828A8389
:202B4E00E0A3F5F0E0C5F045F06007748075F0008003E4F5F07F001201D112006A4B7F0080
:202B6E001201D1F07F011201D1E0A3F5F0E0C5F0C333C5F033C5F0790B7AA512007CE4F575
:202B8E00F089828A83F0A3C5F0F0C5F0022AFD78F9120048E60886F02408C5F03400C5F010
:202BAE007F011201D112006EC39BC5F09CC5F0FBACF07F001201D1E075F0001201197F00D5
:202BCE001201D1F074C075F0A2C0E0C0F0748575F048C0E0C0F07F001201D1E075F000C02A
:202BEE00E0C0F0740375F000123E457FFA12005474C075F0A2C0E0C0F0120CFE1581158114
:202C0E0078F9120048E60886F02408C5F03400C5F018F608A6F0022A92740A75F000C0E0C0
:202C2E00C0F0120B9A158115817F030201EB748A75F048C0E0C0F0120CFE1581158174C00C
:202C4E0075F0A2C0E0C0F074A075F048C0E0C0F0E51475F000C0E0C0F0E517C0E0C0F0E51F
:202C6E003075F000C0E0C0F090A50AE075F000C0E0C0F0740675F000123E457FF412005440
:202C8E0074C075F0A2C0E0C0F0120CFE1581158174C075F0A2C0E0C0F074D875F048C0E02F
:202CAE00C0F0E51575F000C0E0C0F07403123E457FFA12005474C075F0A2C0E0C0F0120C13
:202CCE00FE1581158174C075F0A2C0E0C0F074E675F048C0E0C0F0E51675F000C0E0C0F02A
:202CEE00E522C0E0C0F0E51A75F000C0E0C0F07405123E457FF612005474C075F0A2C0E0F7
:202D0E00C0F0120CFE1581158174C075F0A2C0E0C0F0741175F049C0E0C0F0E52475F00031
:202D2E00C0E0C0F0E525C0E0C0F0E52675F000C0E0C0F0E527C0E0C0F0740675F000123E90
:202D4E00457FF412005474C075F0A2C0E0C0F0120CFE1581158174C075F0A2C0E0C0F07475
:202D6E004575F049C0E0C0F0E52475F000C333C5F033C5F0797B7AA412007C89828A83E069
:202D8E00A3F5F0E0C0F0C0E0740375F000123E457FFA12005474C075F0A2C0E0C0F0120C74
:202DAE00FE1581158174C075F0A2C0E0C0F0745875F049C0E0C0F0E52575F000C333C5F06C
:202DCE0033C5F0797B7AA412007C89828A83E0A3F5F0E0C0F0C0E0740375F000123E457FBD
:202DEE00FA12005474C075F0A2C0E0C0F0120CFE1581158174C075F0A2C0E0C0F0746A75B4
:202E0E00F049C0E0C0F0E52875F000C0E0C0F0E529C0E0C0F0E52A75F000C0E0C0F0E52B27
:202E2E00C0E0C0F0740675F000123E457FF412005474C075F0A2C0E0C0F0120CFE15811595
:202E4E008174C075F0A2C0E0C0F0749E75F049C0E0C0F0E52875F000C333C5F033C5F079CA
:202E6E009B7AA412007C89828A83E0A3F5F0E0C0F0C0E0740375F000123E457FFA120054FD
:202E8E0074C075F0A2C0E0C0F0120CFE1581158174C075F0A2C0E0C0F074B175F049C0E053
:202EAE00C0F0E52975F000C333C5F033C5F0799B7AA412007C89828A83E0A3F5F0E0C0F07E
:202ECE00C0E0740375F000123E457FFA12005474C075F0A2C0E0C0F0120CFE1581158174AD
:202EEE000A75F000C0E0C0F0120B9A15811581E4F527F52B2290000075F014C2AFC297C24B
:202F0E008CC28D758C4C758A00D28C108D0C30B5FA108D1620B5FAA380F1758C4C758A00B4
:202F2E00B297209813D5F0E9800E758C4C758A00B297209803D5F0D38583F0E58290A90BA8
:202F4E00F0A3E5F0F0D297D28DD2AF90A90BE0A3F5F0E0C5F0227FFC7EFF1201ED78FB12E2
:202F6E000048E60886F018F608A6F074C275F049C0E0C0F0120CFE1581158174C075F0A234
:202F8E00C0E0C0F074E175F049C0E0C0F0747075F094C0E0C0F074A075F00FC0E0C0F07407
:202FAE006475F000C0E0C0F07405123E457FF612005474C075F0A2C0E0C0F0120CFE1581C4
:202FCE001581740E75F04AC0E0C0F0120CFE15811581120399122F037F001201D1F0A3C5D7
:202FEE00F0F0C5F012035745F060030231D474C075F0A2C0E0C0F0742C75F04AC0E0C0F0F9
:20300E007F001201D1E0A3F5F0E0C0F0C0E0740375F000123E457FFA12005474C075F0A21C
:20302E00C0E0C0F0120CFE158115817F001201D1E0A3F5F0E0C5F07BA07C8C12017F700362
:20304E0002308C74C075F0A2C0E0C0F0743575F04AC0E0C0F074A075F08CC0E0C0F07403A5
:20306E0075F000123E457FFA12005474C075F0A2C0E0C0F0120CFE158115810231CA7F001A
:20308E001201D1E0A3F5F0E0C5F07B407C9C12018D70030230DF74C075F0A2C0E0C0F0744B
:2030AE004475F04AC0E0C0F0744075F09CC0E0C0F0740375F000123E457FFA12005474C036
:2030CE0075F0A2C0E0C0F0120CFE158115810231CA746E75F08C7F021201D1F0A3C5F0F0D6
:2030EE00C5F07F021201D1E0A3F5F0E0C5F07B727C9C12018570250231BA7F021201D1E047
:20310E00A3F5F0E0C5F02464C5F03400C5F07F021201D1F0A3C5F0F0C5F080C67F00120134
:20312E00D1E0A3F5F0E0C5F07F021201D112006E120195601F7F021201D1E0A3F5F0E0C535
:20314E00F02464C5F03400C5F07F001201D112006E12019545F0700302317C742A75F00066
:20316E00C0E0C0F0120B9A158115810231B77F021201D1E0A3F5F0E0C5F07B3E7C941201E6
:20318E006E70030231A7747C75F000C0E0C0F0120B9A158115810231B7742075F000C0E05B
:2031AE00C0F0120B9A15811581023108745275F04AC0E0C0F0120CFE158115811203574575
:2031CE00F07003022FE01203BB745575F04AC0E0C0F0120CFE158115817F040201EB90A9E3
:2031EE000D7918C2AFC297C28CC28D758C00758A00D28C30B20C308DFAC28DB29720984920
:20320E0080F1C28C758C00758A00D28CC28D208D3830B2FAE58C858AF0B58CF8B403028091
:20322E00D240D0C5F0F0A3E5F0F0A3208D1B20B2FAE58C858AF0B58CF8C5F0F0A3E5F0F0A4
:20324E00A3208D0530B2FAD9E2D297D2AF227FF57EFF1201ED747975F04AC0E0C0F0120C6D
:20326E00FE1581158174A775F04AC0E0C0F0120CFE1581158174D375F04AC0E0C0F0120C50
:20328E00FE15811581740D75F0A9C0E0C0F0E4C0E0C0E0743275F000C0E0C0F0123F6E7F5A
:2032AE00FA1200541203991231EC12035745F06018E4F5F0790D7AA912007C89828A83E0B2
:2032CE00A3F5F0E0C5F012014C45F06003023BF074187F001201D1F07F001201D1E075F018
:2032EE00007B017C0012018D70120233817F001201D1E0147F001201D1F080DC7F00120158
:20330E00D1E075F000C333C5F033C5F0790D7AA912007C7F001201D1E075F000C333C5F06C
:20332E0033C5F0C001C002790D7AA912007C7F001201D1E0C3940175F000C333C5F033C53A
:20334E00F0C001C002790D7AA912007CD083D082E0A3F5F0E0C5F089828A8312006EC39B1D
:20336E00C5F09CC5F0D083D082F0A3C5F0F0C5F00232FBE47F001201D1F07F001201D1E0FE
:20338E0075F0007B197C0012017F70120235B67F001201D1E0047F001201D1F080DC78FB40
:2033AE00120048E60886F07B037C00120168700302344574C075F0A2C0E0C0F074F175F089
:2033CE004AC0E0C0F07F001201D1E075F000C0E0C0F07F001201D1E075F000C333C5F033C7
:2033EE00C5F0790D7AA912007C89828A83E0A3F5F0E0C0F0C0E07F001201D1E075F000C3B8
:20340E0033C5F033C5F0790D7AA912007C89828A83E0A3F5F0E0C0F0C0E0740575F00012F7
:20342E003E457FF612005474C075F0A2C0E0C0F0120CFE158115817F001201D1E075F000A5
:20344E00C333C5F033C5F0790D7AA912007C89828A83E0A3F5F0E0C5F0C333C5F033C5F0EC
:20346E007F051201D1F0A3C5F0F0C5F07F051201D1E0A3F5F0E0C5F0240CC5F03400C5F0B6
:20348E007B197C001200D87F051201D1F0A3C5F0F0C5F07F001201D1E075F000C333C5F07C
:2034AE0033C5F0790D7AA912007C89828A83E0A3F5F0E0C5F02464C5F03400C5F07BC87CE5
:2034CE00001200D87F071201D1F0A3C5F0F0C5F07F001201D1E075F000C333C5F033C5F062
:2034EE00790D7AA912007C7F051201D1E0A3F5F0E0C5F07F071201D112006E2BC5F03CC557
:20350E00F089828A8312006E2BC5F03CC5F089828A83F0A3C5F0F0C5F078FB120048E60884
:20352E0086F07B037C0012016870030235B374C075F0A2C0E0C0F0740B75F04BC0E0C0F02B
:20354E007F001201D1E075F000C333C5F033C5F0790D7AA912007C89828A83E0A3F5F0E08B
:20356E00C0F0C0E07F001201D1E075F000C333C5F033C5F0790D7AA912007C89828A83E083
:20358E00A3F5F0E0C0F0C0E0740475F000123E457FF812005474C075F0A2C0E0C0F0120C6D
:2035AE00FE1581158102339DE4F5F0790D7AA912007C89828A83E0A3F5F0E0C5F07B087CED
:2035CE00001200BE7F051201D1F0A3C5F0F0C5F07F051201D1E0A3F5F0E0C5F07B0A7C0052
:2035EE001200D87F051201D1F0A3C5F0F0C5F078FB120048E60886F07B017C00120168706A
:20360E000302367674C075F0A2C0E0C0F0741C75F04BC0E0C0F0E4F5F0790D7AA912007CD0
:20362E0089828A83E0A3F5F0E0C0F0C0E07F051201D1E0A3F5F0E0C0F0C0E0740475F000EF
:20364E00123E457FF812005474C075F0A2C0E0C0F0120CFE15811581744675F04BC0E0C04D
:20366E00F0120CFE15811581E4F5F0790D7AA912007C7F051201D1E0A3F5F0E0C5F0898294
:20368E008A83F0A3C5F0F0C5F0E47F021201D1F07F021201D1E075F0007B057C0012017FB1
:2036AE0070120237B57F021201D1E0047F021201D1F080DC7F021201D1E075F000C333C52D
:2036CE00F033C5F079717AA912007CE4F5F0C001C002790D7AA912007C7F021201D1E0247D
:2036EE000175F000C333C5F033C5F02401C5F03400C5F089828A8312006E1200BED083D075
:20370E0082F0A3C5F0F0C5F07F021201D1E075F000C333C5F033C5F079717AA912007C89CB
:20372E00828A83E0A3F5F0E0C5F07B027C0012011989828A83F0A3C5F0F0C5F078FB120040
:20374E0048E60886F07B017C0012016870030237B274C075F0A2C0E0C0F0746375F04BC00C
:20376E00E0C0F07F021201D1E075F000C333C5F033C5F079717AA912007C89828A83E0A338
:20378E00F5F0E0C0F0C0E0740375F000123E457FFA12005474C075F0A2C0E0C0F0120CFE0F
:2037AE00158115810236B378FB120048E60886F07B017C0012016870030237DA746775F07A
:2037CE004BC0E0C0F0120CFE15811581E4F5F07F091201D1F0A3C5F0F0C5F0E47F0112015F
:2037EE00D1F074017F001201D1F07F001201D1E075F0007B197C0012017F60227F001201D4
:20380E00D1E075F000C333C5F033C5F0790D7AA912007C89828A83E0A3F5F0E0C5F045F070
:20382E007012023B847F001201D1E0047F001201D1F080B678FB120048E60886F07B027C3D
:20384E000012016870030238CE74C075F0A2C0E0C0F0746B75F04BC0E0C0F07F001201D197
:20386E00E075F000C0E0C0F07F001201D1E075F000C333C5F033C5F0790D7AA912007C89AA
:20388E00828A83E0A3F5F0E0C0F0C0E0E4F5F079717AA912007C89828A83E0A3F5F0E0C06F
:2038AE00F0C0E0740575F000123E457FF612005474C075F0A2C0E0C0F0120CFE1581158149
:2038CE007F001201D1E075F000C333C5F033C5F0790D7AA912007CE4F5F0C001C002797132
:2038EE007AA912007CD083D082E0A3F5F0E0C5F089828A8312006E12018570030239867F84
:20390E00001201D1E075F000C333C5F033C5F0790D7AA912007C89828A83E0A3F5F0E0C581
:20392E00F045F0700302395E78FB120048E60886F07B027C00120168700302395B747E7533
:20394E00F04BC0E0C0F0120CFE1581158102398378FB120048E60886F07B027C0012016823
:20396E007003023983749075F04BC0E0C0F0120CFE158115810238337F001201D1E075F0A7
:20398E0000C333C5F033C5F0790D7AA912007C740875F000C001C00279717AA912007CD080
:2039AE0083D082E0A3F5F0E0C5F089828A8312006E12018D70030239EF78FB120048E60897
:2039CE0086F07B027C0012016870030239EC749A75F04BC0E0C0F0120CFE158115810238C5
:2039EE003374017F021201D1F07F021201D1E075F0007B047C0012017F7012023B5C7F02E9
:203A0E001201D1E0047F021201D1F080DC7F001201D1E075F000C333C5F033C5F0790D7AE4
:203A2E00A912007C7F021201D1E075F000C333C5F033C5F0C001C00279717AA912007CD016
:203A4E0083D082E0A3F5F0E0C5F089828A8312006E1201857003023B597F001201D1E07595
:203A6E00F000C333C5F033C5F0790D7AA912007C89828A83E0A3F5F0E0C5F0C333C5F0338B
:203A8E00C5F07F031201D1F0A3C5F0F0C5F07F021201D1E02401FB7F031201D1E0A3F5F0DD
:203AAE00E0C5F07C001200D87F031201D1F0A3C5F0F0C5F078FB120048E60886F07B027C80
:203ACE00001201687003023B2374C075F0A2C0E0C0F074B075F04BC0E0C0F07F021201D176
:203AEE00E0240175F000C0E0C0F07F031201D1E0A3F5F0E0C0F0C0E0740475F000123E458E
:203B0E007FF812005474C075F0A2C0E0C0F0120CFE158115817F091201D1E0A3F5F0E0C56E
:203B2E00F07F031201D112006E2BC5F03CC5F07F091201D1F0A3C5F0F0C5F07F011201D113
:203B4E00E0047F011201D1F0023B5C023A0C78FB120048E60886F07B027C00120168700326
:203B6E00023B81740A75F000C0E0C0F0120B9A158115810238337F091201D1E0A3F5F0E042
:203B8E00C5F07F011201D112006A7C001200D87F091201D1F0A3C5F0F0C5F074C075F0A288
:203BAE00C0E0C0F074D175F04BC0E0C0F07F091201D1E0A3F5F0E0C0F0C0E0740375F00082
:203BCE00123E457FFA12005474C075F0A2C0E0C0F0120CFE1581158112035745F07003027A
:203BEE0032931203BB7F0B0201EBE4F5F090A97FF0A3C5F0F0C5F0E4F5F090A97DF0A3C565
:203C0E00F0F0C5F0E4F5F0F53185F032748675F00190A97BF0A3C5F0F0C5F022E53185327B
:203C2E00F012014C45F0600A90A97FE0A3F5F0E0C5F045F07003023CFE90A97DE0A3F5F0D1
:203C4E00E0C0F0C0E01228021581158145F06003023CFE90A981E054047003023CB374C060
:203C6E0075F0A2C0E0C0F074EB75F04BC0E0C0F090A97DE0A3F5F0E0C0F0C0E090A97DE09C
:203C8E00A3F5F0E0C0F0C0E0740475F000123E457FF812005474C075F0A2C0E0C0F0120C66
:203CAE00FE1581158190A97DE0A3F5F0E0C5F012012B90A97DF0A3C5F0F0C5F090A97FE0A0
:203CCE00A3F5F0E0C5F090A97D12006E1201857003023CEFE4F5F090A97DF0A3C5F0F0C5CF
:203CEE00F090A97BE0A3F5F0E0C5F0F53185F0322274FE75F04BC0E0C0F0120CFE158115ED
:203D0E008174C075F0A2C0E0C0F0741575F04CC0E0C0F090A97FE0A3F5F0E0C0F0C0E0901F
:203D2E00A97DE0A3F5F0E0C0F0C0E0E5318532F0C0E0C0F090A97BE0A3F5F0E0C0F0C0E05E
:203D4E00740675F000123E457FF412005474C075F0A2C0E0C0F0120CFE15811581227FFE96
:203D6E007EFF1201ED1201F81220DE120205D2AF120893123BF890A38BE06003023DBD74A0
:203D8E004F75F04CC0E0C0F0120CFE15811581748875F04CC0E0C0F0120CFE1581158174C4
:203DAE008D75F04CC0E0C0F0120CFE158115811212BF740175F00045F07003023E1FE4A2D5
:203DCE001792E0F51F7003023DE0B297B297B297C21712278E122930123C2A120FD17F00D7
:203DEE001201D1F0A3C5F0F0C5F07B007C001201767003023E1C7F001201D1E0A3F5F0E0EA
:203E0E00C0F0C0E0121823158115811212BF023DC074B575F04CC0E0C0F0120CFE158115F8
:203E2E00817F020201EB23F42581F81201B91240E91201B902045E23F42581F8868208864D
:203E4E0083080240E9000000000000000000202020202000000000000000000000000000FE
:203E6E000000000000600101010101010101010101010101011818181818181818181801D4
:203E8E000101010101010A0A0A0A0A0A0202020202020202020202020202020202020202AA
:203EAE000101010101010C0C0C0C0C0C040404040404040404040404040404040404040456
:203ECE000101010100C2D578FB120048E6903E53C2E79355F060027401A2D575F00092F0AF
:203EEE0065F075F0002278FB120048E6A2E7B3E4F5F092E02275F00280CB75F00480C675B6
:203F0E00F00680C175F01680BC75F01780B775F05780B2D2D575F05780AD75F01080A67564
:203F2E00F00880A175F001809C75F020809778FB120048E6C0E008E6C0E0123F0813D0F02F
:203F4E00D0E0500224E02278FB120048E6C0E008E6C0E0123F0313D0F0D0E050E9242022D4
:203F6E0078F7120048868208868308860708088603088604EB4C600AEFF0A31BBBFFF51C88
:203F8E0080F22278FB1200488682088683E4FBFCFFE0A3B42D030FE0A3C39430B40A005031
:203FAE0012FA740A75F0001200BE2AFBE5F03400FC80E4EB8CF0DF030201432278F9120072
:203FCE00488682088683E0600DA380FA78F91200488682088683088601088602C9C582C92C
:203FEE00CAC583CAE0A3C9C582C9CAC583CAF06003A380E8E5828583F02278FB120048866D
:20400E0082088683E4F5F0FAE06009A30ABA00F805F080F4EA2278FB120048E60886F030BE
:20402E00F73A02014378F91200488603088604088605088606ED8EF012019B401CED8EF00E
:20404E002278F91200488603088604088605088606ED8EF012019B40E4EB8CF02278FB12D8
:20406E000048860308860485FEF0E5017F0012017F600575F001E422EF0FF5F0A412017F7B
:20408E0070F6EF1475F0002278F912004886820886830886F0E0B5F0068583F0E58222A311
:2040AE0070F3F5F02278F91200488682088683088601088602C9C582C9CAC583CAE0F5F00B
:2040CE00A3C9C582C9CAC583CAE0B5F0056009A380E37401500274FF02008C12423086822D
:2040EE0008868308E4FEFFE07006124230E4F022B42551A3E0B42D05430780A3E0B4300321
:20410E0043074024D0B40A00500BCE75F00AA42EFEA3E080EEE0B46413E60886F030F7085E
:20412E00430720120143A6F018F68003B4750543070A8021B478054307108019B46F1043CD
:20414E0007088011124230F0A3124230A38095B462624307027A00C004C005C006C007AB5F
:20416E000753031F7C00E60886F01200D8A6F018F6EDD007D006D005D0042430B43A004082
:20418E00022407C0E00AE645F070CC124230A902EF30E505742DF0A30A124239D0E0F0A39D
:2041AE00D9FA0808EF30E7A1EAC39E509C7420F0A30A80F4B4630DAA01124230124239E6C5
:2041CE00F0A380DEB47331C082C08386820886837A00E06004A30A80F98683188682124289
:2041EE0030124239124230E0A31242306004F0A380F2D005D00480AAB4691B86017A00E70D
:20420E006004090A80F91242301242398601E76091F009A380F8F97A01124230124239E9AE
:20422E00809ECDC583CDCCC582CC22EE601A8FF020F715C002EAC39E500C742030F60274C3
:20424E0030F0A30A80EFD002224952302000DF42436F6E736F6C65207374617475732066F7
:20426E006C61677320253032780A00205472616E733A20204865616420253032782C20548D
:20428E0061696C20253032782C2043747220253032782C204D617820253032780A0020521A
:2042AE0065633A202020204865616420253032782C205461696C20253032782C2043747273
:2042CE0020253032782C204D617820253032780A00303132333435363738394142434445BA
:2042EE0046003030200020002A2A2A2042616420636865636B73756D3A202532780A002A55
:20430E00000A002A2120004F4B0A003E002A2A2A204E6F20616464726573732073747269F5
:20432E006E672E2E2E0A004E657420616464726573732069732025730A004E65742061640F
:20434E006472657373205B25735D002E2020537461636B207573656420253032782F2530E6
:20436E0032782E0A004572726F7220666C61677320253032782E20204E6574776F726B207F
:20438E00636865636B73756D206572726F72732025750A004C6F6767696E67206D6F6465AF
:2043AE002069732025750A004E6574206D6F64652069732025750A002A2A2A204E20636DA7
:2043CE00642073796E746178206572726F720A002A2A2A20556E6B6E6F776E20636F6D6DF6
:2043EE00616E643A205B25735D0A00426164676520726573706F6E73652064656C61792017
:20440E006973202575207469636B730A002A2A2A204261642043616C6962726174652063E1
:20442E006F6D6D616E640A002A2A2A20426164676520706F6C6C696E6720696E74657276AA
:20444E00616C20666F7263656420746F2025750A00426164676520706F6C6C696E672069B6
:20446E006E74657276616C206973202575207469636B730A002A2A2A204F75747075743ACB
:20448E002020626164206269742049440A002A2A2A204F75747075743A202062616420663B
:2044AE006F726D61740A004E756D626572206F66206261646765732069732025750A002AF3
:2044CE002A2A2051756572793A202062616420706172616D0A0045534554002A2A2A205544
:2044EE006E6B6E6F776E20636F6D6D616E640A002A2A2A204E6F742073656E740A002A2A03
:20450E002A204D697373696E6720706172616D657465720A00417661696C61626C6520637A
:20452E006F6D6D616E6473202876616C75657320696E20646563696D616C20756E6C657379
:20454E0073206E6F746564290A00202874696D657320696E20352E3136206D7320746963C2
:20456E006B73290A0020413D737472696E6720202B20736574206E6574776F726B20616401
:20458E0064726573730A002042206E2020202020202020207365742062616467652072657C
:2045AE0073706F6E73652074696D652064656C61790A00204352206E20202020202020200A
:2045CE0073686F77204D43313435303330206F736320706572696F642C206E203D20726519
:2045EE00706F72742064657461696C0A002043542020202020202020202063616C696272E7
:20460E00617465207472616E736D6974206F7363696C6C61746F72202855312E3131207472
:20462E006F205431290A0020442020202020202020202A2064756D7020696E7465726E6190
:20464E006C20737461747573207661726961626C65732028736F6D6520696E2068657829C2
:20466E000A0020452020202020202020202A2073686F7720616E6420636C65617220657221
:20468E00726F7220666C6167730A002049206E202020202020202020736574206261646771
:2046AE006520706F6C6C696E6720696E74657276616C0A00204C206E2020202020202020E9
:2046CE0020736574207265706F7274696E67206D6F646520286269746D6170706564290A70
:2046EE0000204E206E2020202020202A2B20736574206E6574776F726B206D6F64650A0036
:20470E002050206E202020202020202020736574206E756D626572206F6620626164676570
:20472E007320746F20706F6C6C0A002051202020202020202020202064756D7020616C6C34
:20474E0020726563656976656420495220494420636F64657320696E206865780A00205177
:20476E00206E20202020202020202064756D702073696E676C6520494420696E2062696E28
:20478E006172790A002051206E2D6E2020202020202064756D702072616E6765206F662043
:2047AE0049447320696E206865780A0020524553455420202020202020706572666F726D07
:2047CE0020706F7765722D6F6E20726573657420696E697469616C697A6174696F6E0A001F
:2047EE002053206E20202020202020202073656E6420495220494420636F6465206E0A0025
:20480E002B206D61726B73206E6574776F726B2D6F6E6C7920636F6D6D616E64730A002A62
:20482E00206D61726B7320646562756767696E6720636F6D6D616E64730A0054726E20256B
:20484E0075205B25303478206865785D0A00526376202575205B25303478206865785D0A60
:20486E000020253033753D25750A0020253033752D253033753D0025303278004952206985
:20488E006E74657266616365207374617475733A0A00204952537461746520253032782CB3
:2048AE0020495265635374617420253032782C204261646765446C792025752C2042616457
:2048CE0067655273702025750A0020495243747220253032782C2000494E756D53656E64B3
:2048EE0020253032782C204952426974733020253032782C2054305469636B73202530324E
:20490E00780A00205472616E733A20204865616420253032782C205461696C2025303278DF
:20492E002C2043747220253032782C204D617820253032782C20005B494F757448656164AA
:20494E005D2D3E253034782C20005B494F75745461696C5D2D3E253034780A0020526563C1
:20496E003A202020204865616420253032782C205461696C20253032782C2043747220252F
:20498E003032782C204D617820253032782C20005B49496E486561645D2D3E20253034789C
:2049AE002C20005B49496E5461696C5D2D3E2025303478002D2D2D20436F6E6E656374203E
:2049CE005531312E3120746F20543120696E7075740A00202020202043656E74657220256B
:2049EE007520487A2C2072616E676520257520487A2C20737465702020257520487A0A008F
:204A0E0020202020507265737320616E79206B657920746F20717569742E2E2E0A00253655
:204A2E007520487A205B003C3C3C20756E6465722025755D0A006F766572202575203E3E71
:204A4E003E5D0A005D0A002D2D2D20446973636F6E6E656374205531312E312066726F6D81
:204A6E0020543120696E7075740A002D2D2D20547269676765722072656D6F746520756EFF
:204A8E00697420666F722065616368206D6561737572656D656E740A0020202020204D4313
:204AAE0031343530333020636C6F636B2069732031362F28626974206672616D652074694E
:204ACE006D65290A0020202020507265737320616E79206B657920746F20717569742E2E23
:204AEE002E0A002053616D706C6520253275207261773D253034783D2535752000637674E1
:204B0E003D253034783D2535752075730A002045737420626974206672616D652061646A06
:204B2E0075737465642066726F6D20257520746F2025752075730A0020426974206672614D
:204B4E006D652074696D65207468726573686F6C64733A20002575200075730A002053616C
:204B6E006D706C652025327520253575207573002C20676C697463682069676E6F726564C7
:204B8E000A002C20756E757365640A002C206C6F6E672073706163652069676E6F726564E3
:204BAE000A002C2025752068616C662D6672616D6573202D3E2025752075732F6672616D6F
:204BCE0065200020426974206672616D652074696D652069732025752075730A00506F6C16
:204BEE00202575205B25303478206865785D0A00426164676520706F6C6C696E67207374B6
:204C0E00617475733A0A0020506F6C4E756D4944732025752C20506F6C4E6578744944208D
:204C2E0025752C20506F6C6C446C792025752C20506F6C6C496E74657276616C2025750A1A
:204C4E00000A49522D4C696E6B204E6574776F726B656420496E667261726564204761748C
:204C6E006577617920436F6E74726F6C6C65722C2056657273696F6E2000312E3062000ADF
:204C8E002020436F70797269676874203139393220436972637569742043656C6C61722C86
:204CAE0020496E632E0A002D2D2D2046656C6C206F75742074686520626F74746F6D210A91
:014CCE0000E5
:00000001FF
